:100000005A2883169B001C141A08552883169A0038
:100010001C1555309D00AA309D009C149C180E287C
:100020001C115528A301A200FF30A207031CA3073F
:10003000031C55280330A100DF3020201428A10123
:10004000E83EA000A109FC30031C2928A0070318E2
:100050002628A0076400A10F262820182F28A01CFE
:1000600033280000332808000310A10CA00CFF3E29
:100070000318342820085528A20003304528A20080
:1000800001304528A20006304528A8002308210297
:10009000031D4C28220820020430031801300319E4
:1000A00002302805031DFF305528831303138312E4
:1000B0006400080083163F308500303095008113BE
:1000C0009F018312073099008316FF23900083124B
:1000D0008B010C100B119001D001831605168516AB
:1000E000831205118316051183120510831605105E
:1000F0008312851083168510831204222321640045
:10010000501A83287D2885207D2805158316051122
:100110008312DD0164000A305D0203189F285D0828
:100120000120D3005D083A3E84000008B20064005C
:100130005308320203199D28A428DD0F8A280130B4
:10014000850683160510831250120130C400C501C4
:100150004408A0004508A1000330A300E8303F2078
:10016000031DBA286400851AB6285016C40A03195C
:10017000C50FA8286400501EBE28A4280130C40062
:10018000C5014408A0004508A1000330A300E830E1
:100190003F20031DD3286400851ACF28A428C40A51
:1001A0000319C50FC1280511831605118312080014
:1001B000DD0164000A305D020318E5285D083A3E5F
:1001C0008400FF308000DD0FD928C401C501C40AB6
:1001D0000319C50A23216400501AFB284408A00013
:1001E0004508A100FD30A300E8303C20031DFA289B
:1001F000E728FB281A290511831605118312DD0152
:1002000064000A305D02031812295D083A3E84003A
:100210000008B2005D0883169B0083123208062096
:10022000DD0F00290130A300F430132005158316DB
:10023000051183120330A300E83013200511831643
:1002400005118312080050126400851E2929080038
:1002500045290C10CA01CB014A088E004B088F00BB
:1002600010146400851A3529312910100E08CA00AF
:100270000F08CB004A08A0004B08A1000130A300E2
:100280005E303C20031D452908004A08A0004B08A9
:10029000A1000430A300E2303C20031D5429E230C9
:1002A000C6000430C70081294A08A0004B08A100FD
:1002B0000A30A3008C303C20031D63298430C60023
:1002C0000330C70091294A08A0004B08A1000C3058
:1002D000A300E4303C20031D7229EE30C60002303A
:1002E000C70091294A08A0004B08A1000C30A300C8
:1002F000E4304220031D8129B030C6000430C7001D
:1003000089296400851E852981296400851A892927
:1003100085296400851E8D2989296400851A912903
:100320008D29DD0164000A305D020318022A0130C4
:10033000DE00640005305E020318002A0C10CA01BA
:10034000CB014A088E004B088F0010146400851EF4
:10035000B129640008300F020318AF29A629B1297A
:10036000D12910100E08CA000F08CB004A08A000BF
:100370004B08A1004708A30046084220031DC929D5
:10038000D2175D083A3E8400520880000310D20C58
:10039000D129D2135D083A3E840052088000031030
:1003A000D20C0C10CA01CB014A088E004B088F00FA
:1003B00010146400851ADE29D929FE2910100E08B0
:1003C000CA000F08CB004A08A0004B08A10047084C
:1003D000A30046084220031DF629D2175D083A3EC5
:1003E0008400520880000310D20CFE29D2135D084D
:1003F0003A3E8400520880000310D20CDE0F992987
:10040000DD0F9229501608006400051E082A262ACE
:100410000130CC00CD014C08A0004D08A1001330E4
:10042000A30088303F20031D1D2A6400051E192AE1
:10043000042ACC0A0319CD0F0B2A051583160511C2
:100440008312D8200511831605118312080063005A
:02045000272A59
:02400E00CC3FA5
:00000001FF
